:020000040000FA
:100000000C94C1010C94E9010C94E9010C940716BD
:100010000C9407160C9407160C94E9010C94E90152
:100020000C94E9010C94E9010C94E9010C94E901A8
:100030000C94E9010C94E9010C94E9010C94E90198
:100040000C94BD150C94E9010C948B150C9465155A
:100050000C94E9010C94E9010C94E9010C94E90178
:100060000C947F160C94E90107634236B79BD8A71E
:100070001A39685618AEBAAB558C1D3CB7CC5763CD
:10008000BD6DEDFD753EF6177231BF000000803F7B
:1000900008000000BE922449123EABAAAA2ABECD97
:1000A000CCCC4C3E00000080BEABAAAAAA3E000009
:1000B0000000BF000000803F000000000008417801
:1000C000D3BB4387D1133D190E3CC3BD4282AD2B38
:1000D0003E68EC8276BED98FE1A93E4C80EFFFBE30
:1000E00001C4FF7F3F00000000004E414E494E49D1
:1000F0005459494E46CDCCCC3D0AD7233C17B7D1F5
:100100003877CC2B329595E6241FB14F0A0000209A
:10011000410000C84200401C4620BCBE4CCA1B0E19
:100120005AAEC59D7400407A10F35A00A0724E1862
:10013000090010A5D4E80000E87648170000E40B99
:1001400054020000CA9A3B000000E1F5050000805F
:10015000969800000040420F000000A086010000B9
:1001600000102700000000E8030000000064000009
:100170000000000A00000000000100000000002C48
:1001800076D888DC674F0823DFC1DFAE59E1B1B70D
:1001900096E5E3E453C63AE651997696E8E6C284DA
:1001A00026EB898C9B62ED407C6FFCEFBC9C9F40F2
:1001B000F2BAA56FA5F490055A2AF75C936B6CF917
:1001C000676DC11BFCE0E40D47FEF520E6B500D0ED
:1001D000ED902E0300943577050080841E08000002
:1001E000204E0A000000C80C333333330F986E12D0
:1001F000831141EF8D2114893BE65516CFFEE6DBD6
:1002000018D1844B381BF77C1D901DA4BBE424201F
:100210003284725E228100C9F124ECA1E53D2754AD
:100220003D0020572F6D5E3220555620496E746573
:100230006E7369747900234E6F20504D2073656E84
:10024000736F7221004E6F2073656E736F722100A1
:100250004C6967687420496E74656E7369747900BF
:10026000495220466C616D65204C6576656C3D0099
:10027000476173206C6576656C3D0023496E76613D
:100280006C6964206B657921000000000024002760
:10029000002A0023626D70206661696C656400232A
:1002A00057656C636F6D6520746F20757365204EA4
:1002B000616E6F204C6F67676572004D533D002380
:1002C0005556207A65726F20766F6C746167652071
:1002D0003D00503D0042543D004448543D002344FD
:1002E00075726174696F6E3D0054494D45443D001F
:1002F00023496E74657276616C3D0054494D4549E1
:100300003D0053484F57533D004C6F67676572205F
:100310004E616D653A20004C4F47474552005645A7
:100320005253494F4E005245424F4F540000000077
:1003300008000201000003040700000000000000A4
:100340000000000000230026002900000000002516
:100350000028002B00040404040404040402020224
:1003600002020203030303030301020408102040F6
:1003700080010204081020010204081020009E17CA
:10038000E41F11241FBECFEFD8E0DEBFCDBF11E0C8
:10039000A0E0B1E0E6E6F9E502C005900D92AE3EC0
:1003A000B107D9F724E0AEEEB1E001C01D92A1384B
:1003B000B207E1F711E0C0ECD1E004C02197FE01E3
:1003C0000E94892ACF3BD107C9F70E9400190C94DB
:1003D000A62C0C940000089508950895AF92BF9242
:1003E000CF92DF92EF92FF920F931F93CF93DF9301
:1003F0006C017B018B01040F151FEB015E01AE1830
:10040000BF08C017D10759F06991D601ED91FC9151
:100410000190F081E02DC6010995892B79F7C5017E
:10042000DF91CF911F910F91FF90EF90DF90CF90D0
:10043000BF90AF900895CF93DF93FC014481558125
:100440006081718181E093E00E94EE01EC0142E065
:1004500050E06AE471E081E093E00E94EE018C0FCD
:100460009D1FDF91CF910895FC01538D448D252F61
:1004700030E0842F90E0821B930B541710F0CF963E
:10048000089501970895FC01918D828D981761F070
:10049000A28DAE0FBF2FB11D5D968C91928D9F5F87
:1004A0009F73928F90E008958FEF9FEF0895FC0166
:1004B000918D828D981731F0828DE80FF11D858D19
:1004C00090E008958FEF9FEF0895FC01918D228DAC
:1004D000892F90E0805C9F4F821B91098F73992731
:1004E000089581E093E00E94650221E0892B09F4E0
:1004F00020E0822F089580E090E0892B29F00E946F
:10050000710281110C9400000895FC01A48DA80FC4
:10051000B92FB11DA35ABF4F2C91848D90E0019645
:100520008F739927848FA689B7892C93A089B18965
:100530008C91837080648C93938D848D981306C006
:100540000288F389E02D80818F7D80830895EF926A
:10055000FF920F931F93CF93DF93EC0181E0888F7D
:100560009B8D8C8D98131AC0E889F989808185FF4D
:1005700015C09FB7F894EE89FF896083E889F989EF
:1005800080818370806480839FBF81E090E0DF91F1
:10059000CF911F910F91FF90EF900895F62E0B8D44
:1005A00010E00F5F1F4F0F731127E02E8C8D8E11FF
:1005B0000CC00FB607FCFACFE889F989808185FF66
:1005C000F5CFCE010E948502F1CFEB8DEC0FFD2F10
:1005D000F11DE35AFF4FF0829FB7F8940B8FEA8921
:1005E000FB8980818062CFCFCF93DF93EC01888D30
:1005F0008823B9F0AA89BB89E889F9898C9185FD9E
:1006000003C0808186FD0DC00FB607FCF7CF8C912B
:1006100085FFF2CF808185FFEDCFCE010E9485025C
:10062000E9CFDF91CF910895833081F028F48130B4
:1006300099F08230A9F008958730A9F08830C9F088
:100640008430B1F4809180008F7D03C08091800060
:100650008F7780938000089584B58F7784BD089547
:1006600084B58F7DFBCF8091B0008F778093B000F1
:1006700008958091B0008F7DF9CFCF93DF93ECE3A5
:10068000F3E08491E8E7F3E0D491E4E6F3E0C49189
:10069000CC23A1F081110E941403EC2FF0E0EE0FA7
:1006A000FF1FEF5BFC4FA591B491EC91ED2381E02E
:1006B00090E009F480E0DF91CF91089580E090E030
:1006C000FACF1F93CF93DF93282F30E0F901E35D3A
:1006D000FC4F8491F901E759FC4FD491F901EB5A91
:1006E000FC4FC491CC23A9F0162F81110E94140352
:1006F000EC2FF0E0EE0FFF1FE55BFC4FA591B491EE
:100700008FB7F894EC91111108C0D095DE23DC93DB
:100710008FBFDF91CF911F910895DE2BF8CFCF933C
:10072000DF9390E0FC01E759FC4F24918B5A9C4FDA
:10073000FC0184918823D1F090E0880F991FFC017F
:10074000E757FD4FA591B491FC01E55BFC4FC591C6
:10075000D49161110EC09FB7F8948C91E22FE0956F
:100760008E238C932881E223E8839FBFDF91CF9172
:1007700008958FB7F894EC91E22BEC938FBFF6CFEE
:100780008E3008F08E502091000190E4299F900156
:1007900011248770822B80937C0080917A00806482
:1007A00080937A0080917A0086FDFCCF809178005A
:1007B0009091790008953FB7F89480917B029091D1
:1007C0007C02A0917D02B0917E0226B5A89B05C057
:1007D0002F3F19F00196A11DB11D3FBFBA2FA92FC0
:1007E000982F8827BC01CD01620F711D811D911DBD
:1007F00042E0660F771F881F991F4A95D1F7089529
:100800008F929F92AF92BF92CF92DF92EF92FF9220
:100810006B017C010E94DB034B015C01C114D1041C
:10082000E104F104B9F00E94DB03681979098A092F
:100830009B09683E73408105910580F321E0C21A4F
:10084000D108E108F10888EE880E83E0981EA11C0B
:10085000B11CE4CFFF90EF90DF90CF90BF90AF90AE
:100860009F908F9008958F929F92AF92BF92EF9238
:10087000FF921F93CF93DF93C82F109275041092AD
:10088000760410927704109278041092790461E053
:100890008FE00E948F0360E08FE00E9461036C2F65
:1008A00070E090E080E00E94000460E08FE00E9431
:1008B0008F038BE990E00197F1F7C0E9D1E00E9446
:1008C0003D03892B71F42197D1F78EEF9FEFDF91D4
:1008D000CF911F91FF90EF90BF90AF909F908F901E
:1008E0000895C0E9D1E00E943D03019719F42197D2
:1008F000D1F7EBCFD8E2C0E810E090E9E92EFF2471
:10090000F3940E943D03892B29F481E0E81AF10851
:10091000C1F7DBCF0E94DB034B015C0180E9E82ECD
:10092000FF24F3940E943D03019729F481E0E81A23
:10093000F108C1F7CACF0E94DB03681979098A0957
:100940009B09693271058105910538F0E12FF0E0CE
:10095000E359FB4F80858C2B8087C69511F41F5F70
:10096000C0E8D15051F690E080E0B1CF8F929F92D5
:10097000AF92BF92CF92DF92EF92FF920F931F93AD
:10098000CF93DF938AE0A82EB12CD0E0C0E0EE2414
:10099000EA9493E0F92E88248A9423E0922ED12CB5
:1009A000C12C10E000E08FE00E94C0030817190777
:1009B00090F1C816D90608F46C018815990568F1FC
:1009C0008E159F0508F47C01C80FD91F65E070E003
:1009D00080E090E00E94000481E0A81AB10819F7B5
:1009E0000C0D1D1DCE01801B910B8E199F098819BE
:1009F000990966E070E00E941529CB01DF91CF9143
:100A00001F910F91FF90EF90DF90CF90BF90AF902C
:100A10009F908F9008958C01D0CF4C01D5CF2FB7E8
:100A2000F8946091770270917802809179029091A8
:100A30007A022FBF08952091740230917502281711
:100A4000390771F49091730280917202981741F006
:100A5000E0917302F0E0EE5CFD4F808190E008953C
:100A60008FEF9FEF08950895EF92FF920F931F93DA
:100A7000CF93DF93DC015C96ED90FC905D97E114E1
:100A8000F10479F481E090E013969C938E93129791
:100A900090E080E0DF91CF911F910F91FF90EF9058
:100AA00008955196ED91FC91529750968C915097E4
:100AB000982F90950FB75E962C915E97122F12701B
:100AC00021FD6095F8942081112319F1282B2083B2
:100AD000E7012197F1F728E0462F50E0308160FFD1
:100AE0001AC0382B3083E7012197F1F7BA017595C9
:100AF0006795215089F7112381F0808189238083B4
:100B00000FBF5C968D919C910197F1F781E090E089
:100B1000C1CF2923DCCF3923E5CF9081892BEFCFBB
:100B200020917402309175022817390771F4809171
:100B300072022091730290E0805C9F4F821B9109AA
:100B400060E470E00E942929089590E080E0089513
:100B5000209174023091750228173907B9F49091E9
:100B6000730280917202981789F0E0917302F0E0AD
:100B7000EE5CFD4F80812091730230E02F5F3F4F8C
:100B80002F7333272093730290E008958FEF9FEF28
:100B900008950F931F930E940F056093560470935E
:100BA000570480935804909359048EE494E00E9473
:100BB000A80597FF1DC00E940F05009156041091D3
:100BC00057042091580430915904601B710B820B1B
:100BD000930B0091520410915304209154043091CE
:100BE00055046017710782079307F8F28FEF9FEFA4
:100BF0001F910F910895E0917402F0917502E8172A
:100C0000F90769F4A389B4899C9185898095892322
:100C10008C93109275021092740281E0089580E026
:100C2000089520910F02260F3327331F21323105FB
:100C3000ECF42091D702FC0190E080E0243069F0D0
:100C400082E00895A0910F022191AC0141515E4FC5
:100C5000A40FB52FB11D2C930196861798F38091A0
:100C60000F02680F60930F0280E0089581E00895FD
:100C70001092D70281E08093D6021092B10261E017
:100C800082E10E94610361E083E10E946103E9EB7C
:100C9000F0E080818E7F808380818D7F808388E4F7
:100CA0008093B80085E48093BC0008951092900270
:100CB00010928F021092DE02109200030E943806FA
:100CC0008BEE91E090938E0280938D028CEE91E0FA
:100CD00090938C0280938B020895CF93DF9391E0E1
:100CE0009093EE018823B9F0C091B800D091BA007A
:100CF0008091BC008A7B8093BC0060E082E10E940E
:100D0000610360E083E10E9461030E943806D09392
:100D1000BA00C093B800DF91CF910895CF92DF92CF
:100D2000EF92FF920F931F93CF93DF93D091000325
:100D300081E0D13208F09CC0C091FF020E94DB0329
:100D40006B017C018091D70281116CC082E080939D
:100D5000D70281E08093D6028FEF8093D502109264
:100D6000D402D093D302AFEDB2E0E3EBF2E080E047
:100D7000D8138DC01092B2028091B202CC0FC82B52
:100D8000C093B2028091B102813009F084C0109208
:100D9000B1020E94DB036B017C018091B20280935F
:100DA000BB008091D9029091DA02A091DB02B09150
:100DB000DC02892B8A2B8B2BA1F00E94DB03009194
:100DC000D9021091DA022091DB023091DC026C1919
:100DD0007D098E099F09061717072807390708F4A8
:100DE00042C08091BC0083FDD8CF85EC8093BC00CD
:100DF0000E94DB036B017C018091D702823009F4F1
:100E00004CC08091D5028F3F09F469C08091D50212
:100E1000803209F466C08091D502803309F463C042
:100E200084E026C08091D9029091DA02A091DB0281
:100E3000B091DC02892B8A2B8B2B09F483CF0E9483
:100E4000DB030091D9021091DA022091DB0230918C
:100E5000DC026C197D098E099F0906171707280700
:100E6000390708F06FCF8091D8020E946D0685E0A7
:100E70001092DE02109200031092DD02DF91CF91FA
:100E80001F910F91FF90EF90DF90CF9008959D916B
:100E900091938F5F6DCF85EEA9CF8091D90290910C
:100EA000DA02A091DB02B091DC02892B8A2B8B2B1A
:100EB00009F4A2CF0E94DB030091D9021091DA025B
:100EC0002091DB023091DC026C197D098E099F09AB
:100ED000061717072807390708F08ECFC4CF80E020
:100EE000C7CF82E0C5CF83E0C3CFCF92DF92EF922E
:100EF000FF920F931F93CF93DF93D82FC62F6132AA
:100F000008F098C00E94DB036B017C018091D7023E
:100F100081116BC081E08093D7028093D6029FEF4E
:100F20009093D5021092D4029C0F9093D302809399
:100F3000B2028091B202DD0FD82BD093B202809121
:100F4000B102813009F078C01092B1020E94DB0337
:100F50006B017C018091B2028093BB008091D90229
:100F60009091DA02A091DB02B091DC02892B8A2BEE
:100F70008B2BA1F00E94DB030091D9021091DA02C1
:100F80002091DB023091DC026C197D098E099F09EA
:100F9000061717072807390708F448C08091BC00D6
:100FA00083FDD8CF85EC8093BC000E94DB036B01EE
:100FB0007C018091D702813009F440C08091D40235
:100FC0008C1710F4C091D402E3EBF2E0A1E9B2E097
:100FD00080E08C1355C08C2FDF91CF911F910F9122
:100FE000FF90EF90DF90CF9008958091D90290917B
:100FF000DA02A091DB02B091DC02892B8A2B8B2BC9
:1010000009F484CF0E94DB030091D9021091DA0227
:101010002091DB023091DC026C197D098E099F0959
:10102000061717072807390708F070CF8091D802F4
:101030000E946D06C0E0CFCF85EEB5CF8091D9027A
:101040009091DA02A091DB02B091DC02892B8A2B0D
:101050008B2B09F4AECF0E94DB030091D9021091D3
:10106000DA022091DB023091DC026C197D098E09D5
:101070009F09061717072807390708F09ACFD6CF18
:1010800091919D938F5FA5CFE091900280918F0207
:10109000E81730F4F0E0EF56FD4F808190E00895BE
:1010A0008FEF9FEF08959091900280918F022FEF24
:1010B0003FEF981748F4E92FF0E0EF56FD4F2081FD
:1010C00030E09F5F90939002C901089580918F0254
:1010D00090919002891B990B0895CF92DF92EF9225
:1010E000FF920F931F93CF93DF937C01CB018A0173
:1010F0002091DD02222389F0EB016B01C40ED51E85
:10110000CC15DD0569F06991D701ED91FC91019055
:10111000F081E02DC7010995F3CF642F0E941106DD
:10112000C801DF91CF911F910F91FF90EF90DF9059
:10113000CF900895CF93DF931F92CDB7DEB7698329
:101140002091DD022223F9F020910003203258F093
:1011500021E030E0FC013383228390E080E00F90B7
:10116000DF91CF9108958091DE02E82FF0E0E15207
:10117000FD4F998190838F5F8093DE0280930003FF
:1011800081E090E0ECCF61E0CE0101960E94110673
:10119000F7CF90E080E00895FC0124813581232B76
:1011A00011F00C941B0208958F929F92AF92BF9200
:1011B000CF92DF92EF92FF92CF93DF93C0E2D4E021
:1011C000988121E02093DD029093FF021092DE02CD
:1011D00010920003682F8EE993E00E949A080E9403
:1011E0008E0663E088810E947507109290028093BA
:1011F0008F028EE993E00E945308092E000CAA0B7F
:10120000BB0B8824982EA92EBA2E8EE993E00E945B
:101210005308092E000CAA0BBB0B6C017D01C828DA
:10122000D928EA28FB28FE2CED2CDC2CCC248EE9D6
:1012300093E00E945308BC01990F880B990B6C290D
:101240007D298E299F29DF91CF91FF90EF90DF902C
:10125000CF90BF90AF909F908F9008958F929F9264
:10126000AF92BF92CF92DF92EF92FF920F931F93B4
:10127000209129042F3F19F48AEF0E94D40800918D
:101280002D0410912E0430E020E0C72ED82EE92E38
:10129000FF24E7FCFA94C01AD10AE20AF30A57E0E5
:1012A00095958795779567955A95D1F7000F111FFA
:1012B000221F331F4B015C01801A910AA20AB30A54
:1012C000A5019401A0912F04B09130040E949D25A6
:1012D0004B015C01FBE0B594A79497948794FA9531
:1012E000D1F7A7019601C701B6010E9405299B010C
:1012F000AC01ACE05595479537952795AA95D1F760
:10130000A0913104B09132040E949D259B01AC0153
:10131000BEE05595479537952795BA95D1F7280D95
:10132000391D4A1D5B1D20932504309326044093EC
:10133000270450932804A5E0B0E00E94922560584D
:101340007F4F8F4F9F4F672F782F892F992787FDCA
:101350009A950E945C2420E030E048EC52E40E9420
:101360007A261F910F91FF90EF90DF90CF90BF9062
:10137000AF909F908F9008952F923F924F925F92DF
:101380006F927F928F929F92AF92BF92CF92DF9295
:10139000EF92FF920F931F93CF93DF93CDB7DEB7FA
:1013A0006B970FB6F894DEBF0FBECDBF0E942E091B
:1013B000809129048F3F39F487EF0E94D4086E8B07
:1013C0007F8B888F998F8091250490912604A0911E
:1013D0002704B09128046C017D01FF0CCC08DC2CA3
:1013E00076019C01AD016C2D7C2D8C2D9C2D345FE4
:1013F00041405109610971098109910929873A8799
:101400004B87652E762E872E982E9B8F5901C42EE2
:10141000D52EE62EF72E082F192F0E943D29322EA9
:10142000232E488B598B6A8B7B8B8C8B9D8B3091B9
:10143000360420913504932F990F990B492F592F7A
:10144000692F792F892F0E943D290CE00E94352AAF
:1014500029833C874A8F5D876E877F87582E492E68
:101460003091380420913704932F990F990BA32CB6
:10147000B22CC888D988EA88FB880C891D89492F35
:10148000592F692F792F892F0E943D2908E00E944A
:101490004E2AA980BC84CA8CDD84EE84FF84052D8D
:1014A000142D0E946B2A70588F4F9F4FE091330488
:1014B000F09134045F01D12CC12CE12CF12C870177
:1014C000E983BA82CB82DC82ED82FE820F831887A9
:1014D000C12CD12CE12CF12C00E010E00E943D2920
:1014E00001E20E944E2A2A8F532E49835C876D8722
:1014F0007E878F87492EA0E00E947D2A09F436C19D
:1015000030913E0420913D04932F990F990BA32C09
:10151000B22CC888D988EA88FB880C891D89492F94
:10152000592F692F792F892F0E943D291901488B46
:10153000598B6A8B7B8B8C8B9D8B30913C042091DB
:101540003B04932F990F990BA984BA84CB84D62C92
:10155000E72CF82C092D1B8D492F592F692F792F36
:10156000892F0E943D2901E10E94352A5101C88836
:10157000D988EA88FB880C891D890E946B2A590149
:101580006A017B01382E192F4E895F89688D798D0C
:1015900084E075956795579547958A95D1F780E0D2
:1015A00090E0A0E1B0E0841B950BA60BB70B3C01CB
:1015B0004D01990C6608762C43019C01AD01662D06
:1015C000762D862D962D0FE10E94352A722E832EC0
:1015D000942E5987B62FA72FF82FE92F30913A0470
:1015E00020913904932F990F990B492F592F692F67
:1015F000792F892F03E20E94352A032D0E946B2A3E
:1016000059016A017B018C01272D382D492D5985FF
:101610006B2F7A2F8F2F9E2F0E94742AE5E3AE2E18
:10162000FCE0BF2EC12CD12CE12CF12C00E010E00D
:101630000E943D29AA8CB52CC980DC84ED84FE84EF
:101640000F85142D0E9497292F873E8749875A8737
:101650006B8779838C879D870DE00E944E2A922E9E
:10166000832E742E652E562E472E382E292E30911D
:10167000440420914304932F990F990BA92CB82C63
:10168000C72CD62CE52CF42C032D122D492F592FC5
:10169000692F792F892F0E943D290E943D2909E158
:1016A0000E944E2AAF84BE84C984DA84EB84F98018
:1016B0000C851D850E946B2A19012A013B014C01F2
:1016C0003091420420914104932F990F990B492F97
:1016D000592F692F792F892F0E943D2903E10E94FC
:1016E0004E2A59016A017B018C019101A201B301CB
:1016F000C4010E946B2A08E00E944E2A59016A0127
:101700007B01E82F192F3091400420913F04932F43
:10171000990F990B492F592F692F792F892F04E0A1
:101720000E94352A0E2F0E946B2A0E94222720E059
:1017300030E040E85BE30E94BB246B960FB6F89460
:10174000DEBF0FBECDBFDF91CF911F910F91FF90F4
:10175000EF90DF90CF90BF90AF909F908F907F9051
:101760006F905F904F903F902F90089560E070E0F1
:10177000CB01E3CFCF93909129049F3F41F5682F90
:101780008091200491E09093DD028093FF021092FB
:10179000DE02109200038EE993E00E949A080E94F4
:1017A0008E0662E0809120040E94750710929002DC
:1017B00080938F028EE993E00E945308C82F8EE930
:1017C00093E00E94530820E03C2F282B392B922FC6
:1017D000832FCF910895AF92BF92DF92EF92FF9245
:1017E0000F931F93CF93DF935C010AEA13E0D0E0DD
:1017F000C0E0F801D1908F017501EC0EFD1EC7010C
:101800000E947C25D81621F06D2DC7010E948425E9
:101810002196CC34D10569F78AEA93E0DF91CF9124
:101820001F910F91FF90EF90DF90BF90AF900895C0
:1018300085ED8093BC008091D9029091DA02A0914D
:10184000DB02B091DC020796A11DB11D23E0B69525
:10185000A795979587952A95D1F72091BC0024FDEF
:1018600003C01092D70208954091D9025091DA0234
:101870006091DB027091DC02452B462B472B69F30C
:101880000097A105B10541F025E32A95F1F7000085
:101890000197A109B109E1CF8091D8020C946D069E
:1018A000FC0180819181009711F00C942C2060E064
:1018B00070E0CB010895FB0144815581FC01248136
:1018C00035812417350778F080819181009759F090
:1018D000FB01608171816115710529F00E94892CDD
:1018E00021E0892B09F020E0822F08950F931F93A8
:1018F000CF93DF938C01EB01FC01808191810097F4
:10190000E1F06881798161157105A9F04281538107
:101910002C813D814217530770F00E94822C8C81EC
:101920009D81F801958384831D821C82DF91CF9174
:101930001F910F9108950E942B2B88819981F801A6
:10194000918380838A819B81938382838C819D8113
:1019500095838483198218821B821A82E5CFCF93E4
:10196000DF93EC0188819981009711F00E942B2B65
:10197000198218821D821C821B821A82DF91CF91EC
:101980000895FC0180819181009711F00C942B2B1C
:1019900008950F931F93CF93DF93EC018881998172
:1019A000009759F02A813B812617370730F081E0F4
:1019B000DF91CF911F910F9108958B016F5F7F4F42
:1019C0000E94B42B009759F0998388831B830A8364
:1019D0002C813D81232B59F7FC011082E8CF80E058
:1019E000E7CFEF92FF920F931F93CF93DF93611591
:1019F000710541F480E0DF91CF911F910F91FF902D
:101A0000EF90089541155105B1F07B01EC010C8177
:101A10001D81040F151FB8010E94C90C882351F3C2
:101A2000288139818C819D81B701820F931F0E948B
:101A3000822C1D830C8381E0DECFFC014481558123
:101A4000608171818AE194E00C94F10CCF93DF9373
:101A5000EC01FB0101900020E9F73197AF01461B33
:101A6000570B0E94F10C811103C0CE010E94AF0CF4
:101A7000CE01DF91CF910895CF93DF93EC01FB016D
:101A800044815581608171810E94F10C811103C0F4
:101A9000CE010E94AF0CCE01DF91CF910895EF925D
:101AA000FF920F931F93CF93DF93EC018B01CB0138
:101AB0000E945A207C01BC01CE010E94C90C8111F8
:101AC0000BC0CE010E94AF0CCE01DF91CF911F91D0
:101AD0000F91FF90EF900895FD82EC82B80188810C
:101AE00099810E945320F0CFFC0111821082138251
:101AF0001282158214820C944F0DEF92FF920F9375
:101B00001F93CF93DF93EC017B018A01BA010E94FE
:101B1000C90C81110BC0CE010E94AF0CCE01DF9128
:101B2000CF911F910F91FF90EF9008951D830C832B
:101B3000B701888199810E94822CF0CFFB0101902E
:101B40000020E9F73197AF01461B570B0C947D0D30
:101B50000F931F93CF93DF93CDB7DEB762970FB686
:101B6000F894DEBF0FBECDBF8C01CB01F80111820E
:101B7000108213821282158214824AE0BE016F5FC6
:101B80007F4F0E946320BE016F5F7F4FC8010E949C
:101B90009E0D62960FB6F894DEBF0FBECDBFDF91EB
:101BA000CF911F910F910895CF93DF93EC01FB012B
:101BB0008617970749F0608171816115710541F0C1
:101BC000448155810E947D0DCE01DF91CF91089512
:101BD0000E94AF0CF9CFFC01118210821382128295
:101BE000158214820C94D40DFC0111821082138290
:101BF000128215821482FB0101900020E9F73197CF
:101C0000AF01461B570B0C947D0DCF92DF92EF92E4
:101C1000FF920F931F93CF93DF936C017B018A0197
:101C20004617570720F48F2D7A01062F182F6CE4E2
:101C300071E0C6010E94F40DC0911204D09113040A
:101C4000EC16FD06F8F40C171D0708F4E801E09106
:101C50000E04F0910F04EC0FFD1F108110826091B3
:101C60000E0470910F046E0D7F1DC6016115710584
:101C700099F00E949E0D80910E0490910F04C80F60
:101C8000D91F1883C601DF91CF911F910F91FF904B
:101C9000EF90DF90CF9008950E94AF0CECCFEF92C1
:101CA000FF920F931F93CF93DF93CDB7DEB7A1972A
:101CB0000FB6F894DEBF0FBECDBF7C01CB01BA01D9
:101CC000F70111821082138212821582148242E07F
:101CD000420F8E010F5F1F4F0E940A20009789F06C
:101CE000BC01C7010E949E0DA1960FB6F894DEBFFD
:101CF0000FBECDBFDF91CF911F910F91FF90EF905D
:101D00000895C7010E94AF0CEFCF8F929F92AF92C0
:101D1000BF92EF92FF920F931F93CF93DF93CDB7B4
:101D2000DEB72C970FB6F894DEBF0FBECDBF64E6CA
:101D300070E080E090E00E940004809104019091A6
:101D400005010B9731F580917A04882309F0F89406
:101D500082E10E9433048C0180917A04882309F087
:101D600078940115110509F4BAC080E090ECA9E758
:101D7000B4EC80936D0490936E04A0936F04B093C1
:101D800070048093710490937204A0937304B093D1
:101D900074048091040190910501469731F580917A
:101DA0007A04882309F0F89481E00E9433048C01BE
:101DB00080917A04882309F078940115110509F4BB
:101DC000EFC080E090ECA9E7B4EC80936D049093B1
:101DD0006E04A0936F04B093700480937104909389
:101DE0007204A0937304B093740464E670E080E01E
:101DF00090E00E940004012B09F060C04091710442
:101E000050917204609173047091740421E0CE01CA
:101E100007960E944F0E6DE471E0CE0101960E947C
:101E2000F40DBE01695F7F4FCE0101960E943C0D0B
:101E300060E571E00E94260DBC018AE194E00E94F9
:101E4000D40DCE0101960E94C10C40916D045091B9
:101E50006E0460916F047091700421E0CE010196D0
:101E60000E944F0EBE016F5F7F4FCE0107960E940A
:101E7000760CCE0101960E94C10C64E571E0CE01A2
:101E800001960E94F40DBE01695F7F4FCE0101965D
:101E90000E943C0D67E571E00E94260D0E941D0D19
:101EA000CE0101960E94C10C64E670E080E090E0F3
:101EB0000E940004CE0107960E94C10C2C960FB61A
:101EC000F894DEBF0FBECDBFDF91CF911F910F9170
:101ED000FF90EF90BF90AF909F908F9008951091DA
:101EE0007504E09076046E2D70E090E080E00E9432
:101EF0005C242DEC3CEC4CEC5DE30E94BB244B01DC
:101F00005C01612F70E090E080E00E945C249B0106
:101F1000AC01C501B4010E940E2660936D0470935C
:101F20006E0480936F049093700400917704F09096
:101F30007804602F6F7770E090E080E00E945C246E
:101F40004B015C016F2D70E090E080E00E945C240A
:101F50002DEC3CEC4CEC5DE30E94BB249B01AC01FE
:101F6000C501B4010E940E2607FD18C060937104DC
:101F70007093720480937304909374041E0D100F79
:101F80001F0D81E090E020917904121302C090E0CF
:101F900080E000271127081B190BFBCE9058E6CFD5
:101FA0001091760400917504609175047091760427
:101FB00076276727762790E080E00E945A242DEC50
:101FC0003CEC4CEC5DE30E94BB2460936D04709389
:101FD0006E0480936F0490937004E0907804F09006
:101FE00077046F2D6F77762F6E2D90E080E00E9442
:101FF0005A242DEC3CEC4CEC5DE30E94BB24F7FC36
:1020000018C060937104709372048093730490936A
:102010007404100F1E0D1F0D81E090E020917904D3
:10202000121302C090E080E000271127081B190B53
:10203000DCCE9058E6CF4F925F926F927F928F9254
:102040009F92AF92BF92CF92DF92EF92FF92CF9387
:10205000DF93CDB7DEB72C970FB6F894DEBF0FBE77
:10206000CDBF0E94BC092B013C010E942E094B01EF
:102070005C016091B6037091B7038091B8039091B1
:10208000B9030E945C2420E030E048EC52E40E9456
:102090007A266B017C010E94BC0920E030E048EC0C
:1020A00052E40E947A26A70196010E947A2621E036
:1020B0003EED42E45EE30E947B276B017C0120E061
:1020C00030E048EC52E4C301B2010E947A26AB0131
:1020D000BC0122E0CE0101960E944F0EBE016F5F4F
:1020E0007F4F82E094E00E94760CCE0101960E9420
:1020F000C10C43E050E063EE71E082E094E00E94A6
:10210000F10C62E074E088E094E00E94D40D62EC8F
:1021100071E0CE0101960E94F40D62E074E0CE0100
:1021200001960E943C0DBC0182E094E00E94D40D17
:10213000CE0101960E94C10C6FE172E08AE194E049
:102140000E944F0D21E0B501A401CE0101960E942D
:102150004F0ECE0101960E941D0DCE0101960E94E8
:10216000C10C45E050E069E571E08AE194E00E942D
:10217000F10CA701960160E070E080E89FE30E9407
:102180000D2620E03AE24DE257E40E94BB24AB0169
:10219000BC0121E0CE0101960E944F0EBE016F5F8F
:1021A0007F4FCE0107960E94EB0D6FE571E0CE01E7
:1021B00007960E94260D0E941D0DCE0107960E94D3
:1021C000C10CCE0101960E94C10C62E074E0CE0108
:1021D00001960E94EB0D6EE971E0CE0101960E941E
:1021E000260D6AE174E00E943C0DBC018AE194E096
:1021F0000E94D40DCE0101960E94C10C65E070E0F2
:1022000080E090E00E9400042C960FB6F894DEBFA8
:102210000FBECDBFDF91CF91FF90EF90DF90CF90B9
:10222000BF90AF909F908F907F906F905F904F90F6
:1022300008952F923F924F925F926F927F928F926A
:102240009F92AF92BF92CF92DF92EF92FF920F9345
:102250001F93CF93DF93CDB7DEB7ED970FB6F8940A
:10226000DEBF0FBECDBF8C016CE471E08AE194E06B
:102270000E949E0DC8010596059740F00C3E2FEF79
:10228000120724F010938202009381020C3F8FEF1B
:10229000180709F478C30CF058C0083FAFEF1A07CD
:1022A000C4F4063FBFEF1B07ECF4053FEFEF1E073A
:1022B0000CF0B7C0013FFFEF1F07A4F4083E1F4F0B
:1022C00009F4FFC36BE772E08AE194E00E944F0DCE
:1022D00009C00B3F8FEF18070CF046C3093F1F4F93
:1022E0000CF468C180911E0490911F04892B71F039
:1022F0006AE174E0CE0101960E94EB0DCE010196D9
:102300000E94CC08CE0101960E94C10C64E670E0E8
:1023100080E090E00E940004ED960FB6F894DEBFD6
:102320000FBECDBFDF91CF911F910F91FF90EF9026
:10233000DF90CF90BF90AF909F908F907F906F90E5
:102340005F904F903F902F9008950330110509F44E
:102350001DC33CF510161106A4F00F3FAFEF1A078E
:102360000CF60D3F1F4F09F0ADCF81E080938A023C
:1023700080918102909182029093850280938402E1
:10238000B1CF0130110509F449C00230110509F03F
:1023900099CF80910101882309F4A4CF0E941B10DA
:1023A000A1CF0A301105B4F4063011050CF09ACF14
:1023B0000430110509F46AC30530110509F082CF14
:1023C00060E772E08AE194E00E944F0D0E94B6043B
:1023D000BC016CC30138110509F074CF8091010173
:1023E0008823B1F00E941B106AE174E0CE010196CF
:1023F0000E94EB0DCE0101960E94CC08CE01019601
:102400000E94C10C64EF71E080E090E00E94000443
:1024100064EF71E080E090E00E9400040E94850E6D
:1024200061CF60E080E10E948F0380918A02811178
:10243000BCC08AE090E0A0E0B0E08AAF9BAFACAF58
:10244000BDAF62E272E08AE194E00E944F0D312C50
:10245000212C18AE19AEC12CD12C760102E310E06C
:10246000812C912C540180E10E94C003092E000CA4
:10247000AA0BBB0B880E991EAA1EBB1E65E070E05E
:1024800080E090E00E9400040150110961F7409043
:10249000D2035090D3036090D4037090D503C5014C
:1024A000B4010E945C2420E030E040EA50E40E9445
:1024B000BB2420E030E040E85AE30E94BB2420E047
:1024C00030E048E452E40E947A26A30192010E947F
:1024D0000D2620E030E040E751E40E94BB244B0190
:1024E0005C01A30192016AE979E989E390E40E9421
:1024F0000D269B01AC01C501B4010E947A2620E0A3
:1025000030E0A9010E940E2620E030E040E251E4D4
:102510000E94BB245B018C01232D322D48AD59ADA7
:102520000E947627181624F43A2C2B2C08AF19AFEA
:102530009FEFC91AD90AE90AF90A8AAD9BADACAD79
:10254000BDAD8C159D05AE05BF050CF087CF6EE1C6
:1025500070E080E090E00E94000422E0432D522DC4
:1025600068AD79ADCE0180960E944F0E61E671E0B4
:10257000CE0101960E94F40DBE01605E7F4FCE0138
:1025800001960E943C0D6AE174E00E943C0DBC0182
:102590008AE194E00E94D40DCE0101960E94C10C04
:1025A000CE0180960E94C10C9DCE83E090E0A0E019
:1025B000B0E043CF0E940F052B013C018EE494E074
:1025C0000E94FB0564E670E080E090E00E94000459
:1025D00010926904109268041092670410926604C5
:1025E00010926504109264048DE991E090936B045D
:1025F00080936A0490915A04963108F047C02DEBFD
:1026000030E030936504209364042BE931E030938B
:102610006704209366042CE231E030936904209330
:1026200068042091680084E0983048F031E09E30E2
:1026300008F430E081E001C0880F3A95EAF7822B78
:10264000809368002DE630E0983050F02BE630E0C3
:102650009E3030F02CE630E0963110F030E020E093
:102660003093620420936104292F30E0983008F001
:10267000B0C081E001C0880F9A95EAF780936304A7
:1026800080916A0490916B040197F1F7809168043E
:1026900090916904892B21F18091740290917502C7
:1026A000A4E08E349A07E1F0009711F00E94FB0538
:1026B00080916C048E7F80936C0410927202109251
:1026C00073028EE494E09093750280937402E0911B
:1026D0006104F0916204808190916304892B80836E
:1026E00064E670E080E090E00E94000418AEB12C37
:1026F000A12CD12CC12CF12CE12C1E01B0E22B0E0F
:10270000311C0E940F056419750986099709683BF9
:102710007B408105910508F071C08EE494E00E9431
:102720009005892B09F44EC08CED95E0A0E0B0E057
:102730008093520490935304A0935404B09355048F
:102740000E94C90597FD3EC082349105C9F78E01EC
:102750000F5F1F4F48010E94C90597FF47C089813D
:102760008D3481F59801235E3F4F90E080E0F801C1
:1027700041918F01840F911DE217F307C1F78E5B22
:102780009F4F2E8D30E0322F22274F8D240F311D89
:1027900082179307B9F4EC80F12CFE2CEE248D8186
:1027A000E80EF11CCE80D12CDC2CCC248F81C80EFD
:1027B000D11CA884B12CBA2CAA248985A80EB11CDE
:1027C000F1E0F8AF62E370E080E090E00E94000486
:1027D00098CF9E3040F42850310981E001C0880F25
:1027E0002A95EAF74BCF2E503109F7CFD4018D93BC
:1027F0004D01A215B30509F0AECFB1CF0E940F0570
:102800006419750986099709683B7B408105910524
:1028100098F488AD882309F49AC062E370E080E000
:1028200090E00E9400048EE494E00E94FB0562E3C5
:1028300070E080E090E0A4C098AD992309F487C0CF
:10284000B501CE0180960E94A80DB601CE018696F4
:102850000E94A80DB701CE01C2960E94A80DBE012C
:102860006E5C7F4FCE018C960E94EB0D65E671E0A9
:10287000CE018C960E94260DBE016A5D7F4F0E949C
:102880003C0D65E671E00E94260DBE01605E7F4F43
:102890000E943C0DBC018AE194E00E94D40DCE015F
:1028A0008C960E94C10CCE01C2960E94C10CCE0132
:1028B00086960E94C10CCE0180960E94C10CB50183
:1028C000CE0180960E94A80DB601CE0186960E9488
:1028D000A80DB701CE018C960E94A80D67E671E0A5
:1028E000CE01C2960E94F40DBE01645D7F4FCE0101
:1028F000C2960E943C0D6EE971E00E94260DBE0159
:102900006A5D7F4F0E943C0D6EE971E00E94260DCA
:10291000BE01605E7F4F0E943C0D67E771E00E9440
:10292000260DBC018AE194E00E94D40DCE01C2962E
:102930000E94C10CCE018C960E94C10CCE018696DD
:102940000E94C10CCE0180960E94C10C66CF65E446
:1029500072E08AE194E00E944F0D66E372E08AE142
:1029600094E00E944F0D59CF80918A02882321F074
:102970008AE194E00E941B0268EC70E080E090E045
:102980000E940004AFCC10928A02ACCC60E572E0E9
:102990008AE194E00E944F0D8BE0E82EF12C10E0CC
:1029A00000E09924939493E2892E9092DD02809224
:1029B000FF021092DE021092000362E083E20E94A6
:1029C00075071092900280938F028EE993E00E9427
:1029D0005308D82EC12C8EE993E00E9453085C0165
:1029E000AC28BD280E948E06B50190E080E00E94D0
:1029F0005A242AE939E949E95FE30E947A260E94CC
:102A0000F3260617170708F48B0162E370E080E0F5
:102A100090E00E940004A1E0EA1AF10831F619A240
:102A200018A21BA21AA21DA21CA24AE0BE016F5F3F
:102A30007F4FC8010E948320BE016F5F7F4FCE0190
:102A400080960E949E0D6DE771E0CE0101960E9476
:102A5000F40DBE01605E7F4FCE0101960E943C0DD9
:102A600060E871E00E94260D6AE174E00E943C0D6E
:102A7000BC018AE194E00E94D40DCE0101960E942F
:102A8000C10CCE0180960E94C10CD1CE81E0809312
:102A900000010E94B6048C0160E672E08AE194E0D5
:102AA0000E944F0D60E074E0601B710BCE01019637
:102AB0000E94A80DCE0101960E941D0DCE01019627
:102AC00071CDF0E0E0E009950DCC1F920F920FB6AA
:102AD0000F9211242F933F934F935F936F937F93A4
:102AE0008F939F93AF93BF93EF93FF9381E093E016
:102AF0000E948502FF91EF91BF91AF919F918F91BD
:102B00007F916F915F914F913F912F910F900FBEE9
:102B10000F901F9018951F920F920FB60F921124CD
:102B20002F938F939F93EF93FF93E0911103F09175
:102B300012038081E0911703F091180382FD1BC0FE
:102B4000908180911A038F5F8F7320911B038217EE
:102B500041F0E0911A03F0E0EF5FFC4F958F809316
:102B60001A03FF91EF919F918F912F910F900FBEBC
:102B70000F901F9018958081F4CF1F920F920FB67F
:102B80000F9211242F933F938F939F93AF93BF93F3
:102B90008091770290917802A0917902B0917A02A7
:102BA0003091760223E0230F2D3758F50196A11DB1
:102BB000B11D209376028093770290937802A093C0
:102BC0007902B0937A0280917B0290917C02A0916D
:102BD0007D02B0917E020196A11DB11D80937B0202
:102BE00090937C02A0937D02B0937E02BF91AF913F
:102BF0009F918F913F912F910F900FBE0F901F903B
:102C0000189526E8230F0296A11DB11DD2CF1F9261
:102C10000F920FB60F9211242F933F934F935F9310
:102C20006F937F938F939F93AF93BF93EF93FF9394
:102C3000E0917402F0917502309749F0A685B7854E
:102C40008585968D91FF14C09C918923A1F4FF91F5
:102C5000EF91BF91AF919F918F917F916F915F9114
:102C60004F913F912F910F900FBE0F901F9018958D
:102C70009C91892361F7A389B4899C91858980956A
:102C800089238C93868997890197F1F7608D718DDF
:102C9000A685B785558538E020E0CB010197F1F78F
:102CA000822F90E095958795282F4C91452309F028
:102CB0002068315091F7868D81FD209580917202B8
:102CC00090E001968F73992730917302381799F02D
:102CD000A0917202B0E0AE5CBD4F2C938093720263
:102CE000828D938D0197F1F7A389B4898C91958991
:102CF000892B8C93ACCF868D8160868FF1CF1F920C
:102D00000F920FB60F9211242F933F934F935F931F
:102D10006F937F938F939F93AF93BF93EF93FF93A3
:102D20008091B900887F803609F44AC0F0F5883276
:102D300009F4A7C018F5803109F49BC0B8F48823C2
:102D400009F4F9C0883009F494C0FF91EF91BF9164
:102D5000AF919F918F917F916F915F914F913F9133
:102D60002F910F900FBE0F901F901895883109F486
:102D700088C0803251F78093D50214C0803409F4A2
:102D80009DC040F48033B9F38833F9F68093D502BF
:102D900085ECB0C0803509F485C0883509F496C04B
:102DA000883499F60E94180CD0CF883909F48CC069
:102DB00038F5883729F050F4883611F0803729F635
:102DC00083E08093D7021092310257C0883809F40B
:102DD0007BC0803919F0803809F0B7CF809131027B
:102DE000803208F071C0E091310281E08E0F809353
:102DF00031028091BB00F0E0EF5EFD4F80833DC06B
:102E0000803B39F0E0F4803A09F479C0883A09F05F
:102E10009CCF84E08093D7021092100210920F0290
:102E2000E0918D02F0918E02099580910F0281113F
:102E30000FC081E080930F021092EF0109C0803C27
:102E400009F4A6CF883C09F4A3CF883B09F07DCFD5
:102E5000E091100281E08E0F80931002F0E0E151CA
:102E6000FE4F80818093BB009091100280910F02F1
:102E700029C08091B2028093BB0085EC8093BC0096
:102E800064CF9091D4028091D302981758F5E091C5
:102E9000D40281E08E0F8093D402F0E0ED54FD4F18
:102EA0008081E9CFE091D40281E08E0F8093D4023B
:102EB0008091BB00F0E0ED54FD4F80839091D402EF
:102EC0008091D3029817C8F285E8D8CFE091D40258
:102ED00081E08E0F8093D4028091BB00F0E0ED542E
:102EE000FD4F80838091D60281115CCF81E0809379
:102EF000B10284EA8093BC001092D70226CF85EC01
:102F00008093BC001092D70280913102803230F45D
:102F1000E0913102F0E0EF5EFD4F108260913102EE
:102F200070E0E0918B02F0918C0281E192E00995D2
:102F3000109231020ACF1092D50234CF10920403BE
:102F40001092030388EE93E0A0E0B0E080930503C5
:102F500090930603A0930703B093080328E131E0A0
:102F6000309302032093010325EC30E030930E03ED
:102F700020930D0324EC30E03093100320930F03D3
:102F800020EC30E0309312032093110321EC30E069
:102F9000309314032093130322EC30E03093160394
:102FA0002093150326EC30E0309318032093170389
:102FB00010921A0310921B0310921C0310921D030F
:102FC0001092A1031092A0038093A2039093A303F5
:102FD000A093A403B093A5032AE231E030939F03AA
:102FE00020939E0310927A04109251041092500480
:102FF0008093520490935304A0935404B0935504C7
:103000008CE391E090934F0480934E0410926504FA
:10301000109264041092670410926604109269047E
:103020001092680410926B0410926A0460916C0410
:103030006E7F6D7F60936C046695617081E0682798
:1030400089E00E94610361E089E00E948F03E2E76A
:10305000F3E0E491E0935E04EEE5F3E0E491F0E068
:10306000EE0FFF1FE55BFC4F8591949190936004F8
:1030700080935F0460E08AE00E948F0380916C047B
:1030800081FD04C061E08AE00E9461038AE08093D0
:103090005A04E3E7F3E0E491E0935B04EFE5F3E047
:1030A000E491F0E0EE0FFF1FEF5BFC4F85919491F0
:1030B00090935D0480935C048FEF80932904809348
:1030C0002A0480932B0480932C046CE471E08AE141
:1030D00094E00E94F40D6CE471E084E194E00E94BD
:1030E000F40D6CE471E08EE094E00E94F40D6CE469
:1030F00071E088E094E00E94F40D6CE471E082E0FD
:1031000094E00E94F40D65E871E08CEF93E00E947A
:10311000F40D6CE871E086EF93E00E94F40D86E117
:1031200090E09093AB038093AA038CE79CE8A1E026
:10313000B0E08093B6039093B703A093B803B09325
:10314000B90381EA97E6A3E3BDEB8093BA039093BA
:10315000BB03A093BC03B093BD0386E696E6A6EA44
:10316000BFE38093BE039093BF03A093C003B093CB
:10317000C10381E08093CA0329E130E03093CC039E
:103180002093CB038093CD0380E090E4ACE1B5E4E1
:103190008093CE039093CF03A093D003B093D10339
:1031A0001092D2031092D3031092D4031092D5033D
:1031B000E6EDF3E080E1DF011D928A95E9F71092D8
:1031C000E6031092E7031092E8031092E9031092CD
:1031D000EA031092EB031092EC031092ED031092AD
:1031E000EE031092EF031092F0031092F10310928D
:1031F000F2031092F3031092F4031092F503089572
:10320000CF93DF93CDB7DEB72C970FB6F894DEBF20
:103210000FBECDBF789484B5826084BD84B58160D3
:1032200084BD85B5826085BD85B5816085BD809191
:103230006E00816080936E00109281008091810009
:103240008260809381008091810081608093810001
:10325000809180008160809380008091B1008460C3
:103260008093B1008091B00081608093B000809124
:103270007A00846080937A0080917A0082608093E3
:103280007A0080917A00816080937A0080917A0040
:10329000806880937A001092C10061E08EE00E9405
:1032A0008F03E0911103F091120382E08083E0919B
:1032B0000D03F0910E031082E0910F03F0911003C3
:1032C0008FEC808310921903E0911503F09116039F
:1032D00086E08083E0911303F09114038081806184
:1032E0008083E0911303F0911403808188608083D0
:1032F000E0911303F0911403808180688083E09152
:103300001303F091140380818F7D808360E08EE051
:103310000E9461030E94560681E08093DD0283E2F1
:103320008093FF021092DE021092000360E18EE9AA
:1033300093E00E949A080E948E068FE39CE9019711
:10334000F1F700C0000068EC70E080E090E00E94BF
:10335000000484E690E090930301809302010E94B0
:103360007C2580937F0285E690E00E947C258093F7
:10337000800200917F0210918002B801012E000CA2
:10338000880B990B0E945C249B01AC010E94CB2707
:10339000811106C00B5011090C30110508F4A9C0A9
:1033A00084E690E00E94EB0B68EC70E080E090E037
:1033B0000E9400046FE972E08AE194E00E944F0DE0
:1033C0006AE174E0CE0101960E94EB0DCE010196F8
:1033D0000E94CC08CE0101960E94C10C0E945606A4
:1033E00064E670E080E090E00E94000486E780934D
:1033F0002004809129048F3F11F40E945606809189
:1034000029048F3F01F58091200491E09093DD0223
:103410008093FF021092DE021092000360ED8EE9AD
:1034200093E00E949A080E948E0661E08091200439
:103430000E9475071092900280938F028EE993E0AC
:103440000E945308F82EF8E5FF1609F47DC063E9E1
:1034500072E08AE194E00E944F0D109201016AE14E
:1034600074E0CE0101960E94EB0DCE0101960E9400
:10347000CC08CE0101960E94C10C98EE892E93E0F3
:10348000992EA12CB12C712C612C2AE2E22EF12C68
:1034900080E0C82E80E0D82E6CE471E0CE01079663
:1034A0000E94F40D10E081E093E00E94650218167E
:1034B00019060CF0D9C01111D7C081E093E00E9429
:1034C00043028A3009F4B1C08D3009F4AEC089835B
:1034D0001A8241E050E0BE016F5F7F4FCE01079638
:1034E0000E94F10C6AE070E080E090E00E9400042D
:1034F000DACF3AEAC32E33E0D32E04E610E0C80157
:103500000E947C25F60181936F010F5F1F4F003BE6
:103510001105A9F78091AA039091AB03909305013F
:10352000809304016CEA73E0CE0101960E94F40DD1
:10353000BE016F5F7F4F8CEF93E00E94760CCE014F
:1035400001960E94C10C30CF88E80E94BA0B90937C
:103550002E0480932D048AE80E94BA0B90933004C5
:1035600080932F048CE80E94BA0B909332048093CE
:1035700031048EE80E94BA0B909334048093330494
:1035800080E90E94BA0B909336048093350482E957
:103590000E94BA0B909338048093370484E90E9408
:1035A000BA0B90933A048093390486E90E94BA0BCF
:1035B00090933C0480933B0488E90E94BA0B90935B
:1035C0003E0480933D048AE90E94BA0B9093400424
:1035D00080933F048CE90E94BA0B9093420480933D
:1035E00041048EE90E94BA0B9093440480934304F3
:1035F000809129048F3F09F040CF8091200491E011
:103600009093DD028093FF021092DE02109200037D
:1036100064EF8EE993E00E949A086FE38EE993E0ED
:103620000E949A080E948E0628CF109183021123CF
:10363000C9F08B859C85892B09F454CF67E971E02B
:10364000CE0101960E94F40DBE01695F7F4FCE014D
:1036500001960E943C0D0E941B02CE0101960E9421
:10366000C10C40CF11E03ECFBE01695F7F4F8EE0BD
:1036700094E00E94760CCE0107960E94C10C6CE487
:1036800071E08AE194E00E949E0D80911204909175
:1036900013048130910509F0AFC06EE074E0CE01F3
:1036A00001960E94EB0D8D819E81892B89F0E98125
:1036B000FA81309769F080818234A9F1BCF48A32B2
:1036C00009F497C0813441F169EA71E0833231F144
:1036D000BE016F5F7F4F8EE094E00E94D40D6AE0E0
:1036E00070E080E090E00E94000429C08136A1F0E3
:1036F00074F4833469F766EA71E08EE094E00E9426
:103700009E0D21E020938A028DEF9FEF16C0823636
:1037100051F0833681F3DCCF60EA71E08EE094E013
:103720000E949E0D0CC063EA71E08EE094E00E945E
:103730009E0D10928A028CEF9FEF0E941911CE010C
:1037400001960E94C10C8EE094E00E94500CCB01C7
:103750000E94191180918A02882309F43EC00E94B8
:103760000F05A50194010E94DC25CA01B9010E9440
:103770005A2420918602309187024091880250910C
:1037800089020E940D2620910A0130910B0140917F
:103790000C0150910D010E9476271816F4F40E9436
:1037A0000F05A50194010E94DC25CA01B9010E9400
:1037B0005A246093860270938702809388029093C4
:1037C000890280918402909185020E9419116AE019
:1037D00070E080E090E00E940004C114D10409F47C
:1037E0005BCE0E947102882309F456CE0E9400002D
:1037F0004FCE6CEA71E092CF049768F56FEA71E002
:10380000CE0101960E94F40DBE016F5F7F4F8EE0E6
:1038100094E00E945B0C182FCE0101960E94C10C0F
:103820001123C9F08091120490911304029788F03B
:10383000E0910E04F0910F04309759F081818033AC
:103840000CF4845EF701E81BF10987FDF395CF01C5
:103850007FCF80E0F6CF6EE074E084E194E00E94D8
:10386000D40D00911404109115040115110571F087
:10387000F80181918F01882349F0082E000C990BE3
:103880000E94712CF80131978083F2CF66E273E0D9
:10389000CE0101960E94740DBE016F5F7F4F84E1DF
:1038A00094E00E945B0C182FCE0101960E94C10C7F
:1038B000112319F0F30109954DCF6EE173E0CE01AC
:1038C00001960E94740DBE016F5F7F4F84E194E00A
:1038D0000E945B0C182FCE0101960E94C10C11238F
:1038E00099F161EB71E0CE0101960E94F40D66EF53
:1038F00073E0CE0101960E943C0DBC018AE194E088
:103900000E94D40DCE0101960E94C10C6BEB71E0B8
:10391000CE0101960E94F40D6AE174E0CE01019699
:103920000E943C0DBC01CE0107960E94EB0DCE011A
:1039300007960E94CC08CE0107960E94C10CCE01CA
:1039400001960E94C10C06CF67E173E0CE0101969B
:103950000E94740DBE016F5F7F4F84E194E00E946E
:103960005B0C182FCE0101960E94C10C112359F057
:1039700069E073E08AE194E00E944F0D8CEF93E0E0
:103980000E941D0DC3CF62E073E0CE0101960E943C
:10399000740DBE016F5F7F4F84E194E00E945B0C69
:1039A000182FCE0101960E94C10C112301F147E0AE
:1039B00050E066E070E0CE0101960E94050EBE0167
:1039C0006F5F7F4F88E094E00E94760CCE010196F5
:1039D0000E94C10C88E094E00E94500C672B19F4FF
:1039E00010928302B7CEF1E0F0938302B3CE6BEF77
:1039F00072E0CE0101960E94740DBE016F5F7F4F91
:103A000084E194E00E945B0C182FCE0101960E9485
:103A1000C10C112309F479C0409112045091130490
:103A20004730510508F496CE66E070E0CE0101966D
:103A30000E94050EBE016F5F7F4F88E094E00E94F8
:103A4000760CCE0101960E94C10C809108049091E1
:103A50000904009709F455C00E94282060930A01C8
:103A600070930B0180930C0190930D0160EF72E055
:103A70008AE194E00E944F0D40910A0150910B01A0
:103A800060910C0170910D0122E0CE0101960E941F
:103A90004F0EBE016F5F7F4FCE0107960E94EB0D68
:103AA0006DEB71E0CE0107960E94260D0E941D0D60
:103AB000CE0107960E94C10CCE0101960E94C10C56
:103AC0006AE174E0CE0101960E94EB0DCE010196F1
:103AD0000E94CC08CE0101960E94C10C0E940F05E5
:103AE000A50194010E94DC25CA01B9010E945A2453
:103AF0006093860270938702809388029093890274
:103B000029CE60E070E0CB01A9CF69EE72E0CE0172
:103B100001960E94740DBE016F5F7F4F84E194E0B7
:103B20000E945B0C182FCE0101960E94C10C11233C
:103B300009F467C0409112045091130447305105B5
:103B400008F408CE66E070E0CE0101960E94050EF2
:103B5000BE016F5F7F4F88E094E00E94760CCE013B
:103B600001960E94C10C809108049091090400976D
:103B700009F443C00E942820609306017093070156
:103B800080930801909309016EED72E08AE194E060
:103B90000E944F0D4091060150910701609108016C
:103BA0007091090121E0CE0101960E944F0EBE01E5
:103BB0006F5F7F4FCE0107960E94EB0D6DEB71E0BA
:103BC000CE0107960E94260D0E941D0DCE0107967C
:103BD0000E94C10CCE0101960E94C10C6AE174E002
:103BE000CE0101960E94EB0DCE0101960E94CC08F9
:103BF000CE0101960E94C10CADCD60E070E0CB011A
:103C0000BBCF69ED72E0CE0101960E94740DBE013A
:103C10006F5F7F4F84E194E00E945B0C182FCE0110
:103C200001960E94C10C112331F146E050E064E09E
:103C300070E0CE0101960E94050EBE016F5F7F4FBE
:103C400088E094E00E94760CCE0101960E94C10C9F
:103C500088E094E00E94500C7093AB036093AA0339
:103C6000709305016093040180910201909103011A
:103C70000E94EB0B6FCD65ED72E0CE0101960E94C4
:103C8000740DBE016F5F7F4F84E194E00E945B0C76
:103C9000182FCE0101960E94C10C112309F44FC0C8
:103CA000409112045091130463E070E0CE0101963C
:103CB0000E94050EBE016F5F7F4F88E094E00E9476
:103CC000760CCE0101960E94C10C68E074E0CE0132
:103CD00001960E94EB0D1F82188641E050E0BE0164
:103CE000695F7F4FCE0101960E94F10C811104C0E3
:103CF000CE0101960E94AF0CBE016F5F7F4F8CEF2B
:103D000093E00E94D40DCE0101960E94C10C009157
:103D10000004109101040115110509F4A5CF01500B
:103D200011096091FC037091FD03A8018CEA93E0F6
:103D30000E94972CF801E455FC4F108295CF62ED5C
:103D400072E0CE0101960E94740DBE016F5F7F4F3D
:103D500084E194E00E945B0C182FCE0101960E9432
:103D6000C10C112309F48AC040911204509113042C
:103D70004031510508F0EECC62E070E0CE010196D2
:103D80000E94050EBE016F5F7F4F88E094E00E94A5
:103D9000760CCE0101960E94C10C8091080490918E
:103DA0000904009799F10E94282020E030E048ECB7
:103DB00052E40E94BB240E94EC266093B6037093E9
:103DC000B7038093B8039093B9038B019C0100590A
:103DD0001F452140310901341C4921053105D0F02E
:103DE0006FEB71E0CE0101960E94F40D68E074E083
:103DF000CE0101960E943C0D65EC71E00E94260DFB
:103E0000BC018AE194E00E94D40D99CD60E070E09D
:103E1000CB01CBCF0E945C2420E030E048EC52E4A0
:103E20000E947A26AB01BC0122E0CE0101960E94DD
:103E30004F0EBE016F5F7F4F8AE194E00E94760CC7
:103E4000CE0101960E94C10C65ED71E0CE01019694
:103E50000E94F40D6AE174E0CE0101960E943C0DCF
:103E600062EE71E00E94260DBC018AE194E00E949E
:103E7000D40DCE0101960E94C10CF6CE67EE71E022
:103E8000CE0101960E94F40DBE016F5F7F4F84E169
:103E900094E00E945B0C182FCE0101960E94C10C89
:103EA000112309F45EC009E110E0212C312C21011D
:103EB00080E10E94C003BC01990F880B990B0E94FE
:103EC0005C249B01AC01C201B1010E940E261B01C2
:103ED0002C016AE070E080E090E00E940004015054
:103EE000110931F720E030E040EA50E4C201B101AD
:103EF0000E94BB2420E030EC4FE754E40E947A2675
:103F000020E030E048EC51E40E947A266093D2032E
:103F10007093D3038093D4039093D50380910201CF
:103F2000909103010E94EB0B6FEB72E08AE194E049
:103F30000E944F0D4091D2035091D3036091D4035E
:103F40007091D50322E0CE0101960E944F0EBE0172
:103F50006F5F7F4FCE0107960E94EB0D6BEE71E015
:103F60002FCE6BEB72E0CE0101960E94740DBE0164
:103F70006F5F7F4F84E194E00E945B0C182FCE01AD
:103F800001960E94C10C112309F4E4CB4091120464
:103F90005091130463E070E0CE0101960E94050E7B
:103FA000BE016F5F7F4F88E094E00E94760CCE01E7
:103FB00001960E94C10C88E094E00E94500C70931E
:103FC000820260938102C6CB86EF93E00E94C10C0F
:103FD0008CEF93E00E94C10C82E094E00E94C10C3F
:103FE00088E094E00E94C10C8EE094E00E94C10C35
:103FF00084E194E00E94C10C8AE194E00E94C10C2B
:104000008CE391E090934F0480934E048EE494E00F
:104010000C94FB05EF920F931F93CF93DF93E8016E
:1040200034E047FD34E1042E000C550B57FF03C06C
:10403000519541955109E32E022F242FAE010E9484
:104040009D20CE01DF91CF911F910F91EF900895A8
:10405000662777270C94FC211F93FC01992788275A
:10406000BC01E89411911032E9F3193010F01E30C0
:10407000C8F31B3251F01D3249F4689406C00E9407
:104080006E20610F711D811D911D119110531A3009
:10409000B0F33EF490958095709561957F4F8F4F6A
:1040A0009F4F1F910895FB01DC0105900D920020A8
:1040B000E1F70895FC0105900020E9F780959095BF
:1040C0008E0F9F1F0895BB274A3031F4992322F4A5
:1040D000BDE2909581959F4F0C948420592F482FD5
:1040E000372F262F660F771F881F991F660F771FA0
:1040F000881F991F620F731F841F951F660F771FFC
:10410000881F991F0895BB27FB015527AA27880FF1
:10411000991FAA1FA41710F0A41B83955051B9F73B
:10412000A05DAA3308F0A95DA193009779F7B111BA
:10413000B1931192CB010C944524A9E0B0E0E3EADD
:10414000F0E20C94AB256A01F22EB02E102FFBE3A7
:10415000AF2EA01608F41BE31F5F012F27E0AE016E
:104160004F5F5F4F0E944C23BC018981982F99704B
:10417000913009F43FC09BE2E1FC04C09E2D917098
:10418000E0FC3AC05E2D5071E82FE87083FF46C016
:1041900084E0911101C083E0EF2DE81B8F1508F03A
:1041A000E0E0D6018E2F20E2552351F1992329F02A
:1041B000D6019C93C60101966C0196012D5F3F4F7D
:1041C000E2FE24C08EE4D6018C9391E411969C9378
:1041D000119712968C93D9018E2F90E281111BC0FA
:1041E000E20FF32FF11D10828EEF9FEF2996ECE086
:1041F0000C94C7259DE2C6CF90E2C4CF2D93815089
:104200008111FCCFCE0ED11CE0E0D0CF8EE6D601DE
:104210008C9391E6DBCF9D938150E0CF482F447083
:1042200082FF3DC084E0911101C083E08F1510F43E
:10423000EF2DE81BD6018E2F20E2552309F199239B
:1042400029F0D6019C93C60101966C0196012D5F61
:104250003F4FE2FE1BC089E4D6018C938EE4119699
:104260008C93119786E412968C93D9018E2F90E24D
:10427000882309F4B5CF9D938150FACF2D938150B7
:104280008111FCCFCE0ED11CE0E0D9CF89E6D6015A
:104290008C938EE611968C93119786E6E4CF9B0162
:1042A00077FF02C030E020E0A1E0B0E0911102C051
:1042B000B0E0A0E0F9013196AE0FBF1F8B2C912C1E
:1042C000BB2009F461C05401EFEFAE1ABE0AAA0D7B
:1042D000BB1DFA161B0619F014F04F2D4A1B511185
:1042E00088C0E3FC59C07601A42FB0E2A1114FC0F1
:1042F000C40ED11C992309F45BC040E0D60111968D
:10430000F60190836D01552309F448C0012F060F73
:104310009A81582F507184FF03C0913309F40150E2
:1043200010160CF047C0093008F008E0EEE2FE2E4F
:104330005B01A01AB10885019194819491082F3FE7
:10434000320729F4D601FC92F60131966F0162170B
:10435000730794F1021713077CF5DB01A21BB30B63
:10436000AA24A394B12CAC0EBD1EAA0DBB1D1196A0
:104370008C9121503109D601119628153905F4F098
:10438000F60180836D01DBCFB12CA12CA0CFF7010A
:10439000B1937F01A150AACF9111B0CFD601942F34
:1043A00050E302C05D9391509111FCCFC40ED11C1B
:1043B00040E0ACCF01E0BACF80E3DBCF62177307F8
:1043C00031F4963388F4953311F4552369F0F601EE
:1043D0008083FD01842F90E2811108C0A40FB11DDC
:1043E0001C9290E080E002CF81E3F1CF9193815065
:1043F000F3CF911183CF8ACFB0E0A0E0E2E0F2E208
:104400000C94AB255C017B016115710519F0DB0192
:104410008D939C9385010F5F1F4FF501D0818D2FE8
:1044200090E00E9424246C01892BB9F5DD32B9F5A6
:104430000F5F1F4FD5011196DC91C1E05801F1E0EB
:10444000AF1AB10843E050E062EF70E0C5010E948E
:104450002D24892B69F5680182E0C80ED11C45E046
:1044600050E06DEE70E0C6010E942D24892B21F4EE
:10447000680197E0C90ED11CE114F10419F0D701CD
:10448000CD92DC9260E070E080E89FEFC111FFC048
:1044900060E070E080E89FE7FAC05801BBCFDB32F4
:1044A00029F485010E5F1F4FF501D181C0E0C6CF11
:1044B00043E050E06AEE70E0C5010E942D24892B94
:1044C000E9F0F80110E000E020E030E0A9015F0130
:1044D000B0ED8B2E8D0E89E08815C8F19C2E689466
:1044E00091F88C2F8870C2FF16C0811102C00F5F37
:1044F0001F4F3196D501DC91C92DE9CFE114F104AC
:1045000029F00E5F1F4FF7011183008360E070E018
:1045100080EC9FE7BCC0882311F001501109A5E091
:10452000B0E00E9492259B01AC01220F331F441F73
:10453000551F280D311D411D511D283999E9390795
:10454000490799E15907A8F2C6609C2ED2CFAEEF79
:104550008A1206C0C3FD3CC09C2E689493F8C9CF54
:10456000DF7DD534A9F580818D3239F4C061DF015A
:104570001296818162E070E006C0DF018B32C1F3E8
:10458000119661E070E080535D01A61AB70A8A3087
:10459000F8F4E0E8CE16ECE0DE065CF4B601660F57
:1045A000771F660F771FC60ED71ECC0CDD1CC80EFA
:1045B000D11C5D01FFEFAF1ABF0A8C9180538A3086
:1045C000A8F1C4FF03C0D194C194D1080C0D1D1DE6
:1045D000C1FF09C0E114F10431F081E0A81AB1086B
:1045E000D701AD92BC92CA01B9010E945A24C3708E
:1045F000C33009F490584B015C0120E030E0A90180
:104600000E945524882309F440C0C1E2D1E017FF7D
:1046100005C0119501951109C9E0D1E06E01B8E11D
:10462000CB1AD10880E2E82EF12C0FC0D501B1CF12
:10463000FE0125913591459154910E191F09C5012F
:10464000B4010E94BB244B015C01D501C4010E15CD
:104650001F0574F72497F594E794CC16DD06A9F7A7
:104660008A2F880F8B2F881F8F3F49F020E030E082
:10467000A901C501B4010E945524811106C082E23E
:1046800090E090937C0480937B04C501B401CDB786
:10469000DEB7ECE00C94C725283008F027E033277C
:1046A000DA01990F311D87FD916000966105710552
:1046B00039F432602E5F3D9330E32A95E1F7089597
:1046C0009F3F30F080387105610509F03C5F3C5F29
:1046D0003D93913008F08068911DDF93CF931F9335
:1046E0000F93FF92EF92192F987F9695E92F969549
:1046F0009695E90FFF27E158FE4F99273327EE24BF
:10470000FF24A701E70105900894079428F4360FC9
:10471000E71EF81E491F511D660F771F881F991F3E
:104720000694A1F70590079428F4E70EF81E491F98
:10473000561FC11D770F881F991F661F0694A1F78A
:104740000590079428F4F80E491F561FC71FD11D66
:10475000880F991F661F771F0694A1F7059007948D
:1047600020F4490F561FC71FD81F990F661F771FC8
:10477000881F0694A9F784911095177041F0D6957B
:10478000C79557954795F794E7941A95C1F7E5E2D1
:10479000F1E068941590159135916591959105908A
:1047A0007FE27395E118F10A430B560BC90BD00950
:1047B000C0F7E10CF11E431F561FC91FD01D7EF428
:1047C000703311F48A95E6CFE894015030F0080F69
:1047D0000AF40027021708F4202F2395022F7A33BA
:1047E00028F079E37D932A95E9F710C07D932A9507
:1047F00089F6069497956795379517951794E1185C
:10480000F10A430B560BC90BD00998F023957E9102
:1048100073957A3308F070E37C932013B8F77E9198
:1048200070617D9330F0839571E37D9370E32A95F9
:10483000E1F71124EF90FF900F911F91CF91DF913D
:10484000992787FD9095089591110C942825803221
:1048500019F089508550C8F70895FB01DC014150DB
:10486000504088F08D9181341CF08B350CF4805EC3
:10487000659161341CF06B350CF4605E861B611130
:1048800071F3990B0895881BFCCFDC01FC01672FA5
:1048900071917723E1F7329704C07C916D93708317
:1048A0006291AE17BF07C8F308950E94972408F4D9
:1048B00081E00895E89409C097FB3EF490958095B7
:1048C000709561957F4F8F4F9F4F9923A9F0F92FD6
:1048D00096E9BB279395F695879577956795B79554
:1048E000F111F8CFFAF4BB0F11F460FF1BC06F5F3A
:1048F0007F4F8F4F9F4F16C0882311F096E911C04C
:10490000772321F09EE8872F762F05C0662371F06C
:1049100096E8862F70E060E02AF09A95660F771F80
:10492000881FDAF7880F9695879597F90895990F5C
:104930000008550FAA0BE0E8FEEF16161706E80769
:10494000F907C0F012161306E407F50798F0621B8A
:10495000730B840B950B39F40A2661F0232B242B5F
:10496000252B21F408950A2609F4A140A6958FEF7E
:10497000811D811D08950E94CE240C9442250E9421
:10498000342538F00E943B2520F0952311F00C943B
:104990002B250C94312511240C9476250E94532547
:1049A00070F3959FC1F3950F50E0551F629FF00182
:1049B000729FBB27F00DB11D639FAA27F00DB11D9B
:1049C000AA1F649F6627B00DA11D661F829F222724
:1049D000B00DA11D621F739FB00DA11D621F839FAB
:1049E000A00D611D221F749F3327A00D611D231F81
:1049F000849F600D211D822F762F6A2F11249F57CF
:104A000050409AF0F1F088234AF0EE0FFF1FBB1FD1
:104A1000661F771F881F91505040A9F79E3F510590
:104A200080F00C942B250C9476255F3FE4F3983EA0
:104A3000D4F3869577956795B795F795E7959F5F3A
:104A4000C1F7FE2B880F911D9695879597F90895CC
:104A500099278827089597F99F6780E870E060E0BC
:104A600008959FEF80EC089500240A941616170607
:104A700018060906089500240A941216130614064F
:104A800005060895092E0394000C11F4882352F0B2
:104A9000BB0F40F4BF2B11F460FF04C06F5F7F4F6A
:104AA0008F4F9F4F089557FD9058440F551F59F051
:104AB0005F3F71F04795880F97FB991F61F09F3F0B
:104AC00079F087950895121613061406551FF2CF34
:104AD0004695F1DF08C0161617061806991FF1CF84
:104AE00086957105610508940895E894BB276627AB
:104AF0007727CB0197F90895F999FECF92BD81BD33
:104B0000F89A992780B50895262FF999FECF1FBAF4
:104B100092BD81BD20BD0FB6F894FA9AF99A0FBEE6
:104B2000019608950E94FE25A59F900DB49F900DBB
:104B3000A49F800D911D11240895B7FF0C94922518
:104B40000E949225821B930B08952F923F924F92C1
:104B50005F926F927F928F929F92AF92BF92CF920D
:104B6000DF92EF92FF920F931F93CF93DF93CDB716
:104B7000DEB7CA1BDB0B0FB6F894DEBF0FBECDBF8E
:104B800009942A88398848885F846E847D848C845F
:104B90009B84AA84B984C884DF80EE80FD800C8168
:104BA0001B81AA81B981CE0FD11D0FB6F894DEBF4B
:104BB0000FBECDBFED010895A1E21A2EAA1BBB1BAB
:104BC000FD010DC0AA1FBB1FEE1FFF1FA217B307D9
:104BD000E407F50720F0A21BB30BE40BF50B661FEF
:104BE000771F881F991F1A9469F7609570958095B3
:104BF00090959B01AC01BD01CF010895A29FB0012A
:104C0000B39FC001A39F700D811D1124911DB29F00
:104C1000700D811D1124911D08955058BB27AA279E
:104C20000E9425260C9442250E94342538F00E94CB
:104C30003B2520F039F49F3F19F426F40C943125DC
:104C40000EF4E095E7FB0C942B25E92F0E945325E9
:104C500058F3BA17620773078407950720F079F4B1
:104C6000A6F50C9475250EF4E0950B2EBA2FA02D09
:104C70000B01B90190010C01CA01A0011124FF2709
:104C8000591B99F0593F50F4503E68F11A16F04004
:104C9000A22F232F342F4427585FF3CF4695379503
:104CA0002795A795F0405395C9F77EF41F16BA0BC8
:104CB000620B730B840BBAF09150A1F0FF0FBB1F76
:104CC000661F771F881FC2F70EC0BA0F621F731FBF
:104CD000841F48F4879577956795B795F7959E3F1C
:104CE00008F0B0CF9395880F08F09927EE0F9795AD
:104CF000879508950E948E260C9442250E943B259C
:104D000058F00E94342540F029F45F3F29F00C94BC
:104D10002B2551110C9476250C9431250E94532596
:104D200068F39923B1F3552391F3951B550BBB27DA
:104D3000AA2762177307840738F09F5F5F4F220F1F
:104D4000331F441FAA1FA9F335D00E2E3AF0E0E816
:104D500032D091505040E695001CCAF72BD0FE2F60
:104D600029D0660F771F881FBB1F261737074807F4
:104D7000AB07B0E809F0BB0B802DBF01FF279358AC
:104D80005F4F3AF09E3F510578F00C942B250C9420
:104D900076255F3FE4F3983ED4F386957795679543
:104DA000B795F7959F5FC9F7880F911D96958795E1
:104DB00097F90895E1E0660F771F881FBB1F621700
:104DC00073078407BA0720F0621B730B840BBA0BBE
:104DD000EE1F88F7E09508950E94F3266894B111BC
:104DE0000C94762508950E945B2588F09F5798F0D3
:104DF000B92F9927B751B0F0E1F0660F771F881FE0
:104E0000991F1AF0BA95C9F714C0B13091F00E94F9
:104E10007525B1E008950C947525672F782F8827A4
:104E2000B85F39F0B93FCCF3869577956795B39520
:104E3000D9F73EF490958095709561957F4F8F4F8F
:104E40009F4F089597FB16F40E9466270C9429271C
:104E5000E894F92F96EBFF2381F01216130614063F
:104E6000440B9395F69587957795679557954040B0
:104E7000FF23B9F71BC099270895882351F4985050
:104E8000D2F7872B762F652F542F432F322F20E018
:104E9000B1F3121613061406440B88233AF09A95C0
:104EA000440F551F661F771F881FCAF755234AF402
:104EB000440F551F11F460FF04C06F5F7F4F8F4F89
:104EC0009F4F880F9695879597F9089590958095AF
:104ED0007095609550954095309521953F4F4F4F77
:104EE0005F4F6F4F7F4F8F4F9F4F08950E949724C2
:104EF00008F48FEF0895FA01EE0FFF1F3096210599
:104F00003105A1F16115710561F48038BFE39B079C
:104F100049F168949038810561F08038BFEF9B07B4
:104F200041F099234AF5FF3FE1053105210519F1CB
:104F3000E8940894E795D901AA2329F4AB2FBE2F52
:104F4000F85FD0F310C0FF5F70F4A695E0F7F73973
:104F500050F019F0FF3A38F49F779F930DD00F90DF
:104F600007FC9058089546F00C94312560E070E0FD
:104F700080E89FE308954FE79F775F934F933F93B8
:104F80002F930E947B282F913F914F915F910E9418
:104F9000BB240C94D8270E949724880B990B089562
:104FA00029F416F00C942B250C9475250C943125BE
:104FB0000E945B25A8F39638A0F707F80F92E894B3
:104FC0002BE33AEA48EB5FE70E94D1240F920F925D
:104FD0000F924DB75EB70F920E94C328E8E6F0E04B
:104FE0000E940A284F915F91EF91FF91E595EE1F86
:104FF000FF1F49F0FE57E0684427EE0F441FFA9563
:10500000E1F74195550B0E943D280F9007FE0C9447
:1050100031280895DF93CF931F930F93FF92EF9260
:10502000DF927B018C01689406C0DA2EEF010E94AA
:10503000CE24FE01E894A591259135914591559195
:10504000A6F3EF010E942526FE019701A801DA943C
:1050500069F7DF90EF90FF900F911F91CF91DF9153
:1050600008959B01AC0160E070E080E89FE30C9440
:105070007A260C942B250C94F7280E945B25D8F3F4
:105080009923C9F3940F511DA3F39150504094F00C
:1050900059F0882332F0660F771F881F91505040D7
:1050A000C1F79E3F51052CF7880F911D9695879566
:1050B00097F908955F3FACF0983E9CF0BB2786952A
:1050C00077956795B79508F4B1609395C1F7BB0FD5
:1050D00058F711F460FFE8CF6F5F7F4F8F4F9F4FFE
:1050E000E3CF0C94762516F00C94F7280C94312518
:1050F00068940C942B250E945B25A8F39923C1F397
:10510000AEF3DF93CF931F930F93FF92C92FDD2749
:1051100088232AF02197660F771F881FDAF720E08F
:1051200030E040E85FEB9FE3883920F0803E38F0C4
:1051300021968F770E940E26E0E9F0E004C00E94DD
:105140000E26EDEBF0E00E940A288B01BE01EC0177
:10515000FB2E6F5771097595771F880B990B0E946D
:105160005C2428E132E741E35FE30E94CE24AF2DC7
:105170009801AE01FF900F911F91CF91DF910E9496
:1051800025260C944225FA01DC01AA0FBB1F9B01C6
:10519000AC01BF5728F4222733274427507820C07A
:1051A000B75190F4AB2F0024469537952795011CF5
:1051B000A395D2F3002071F0220F331F441FB39543
:1051C000DAF30ED00C940D2661307105A0E88A0741
:1051D000B94630F49B01AC01662777278827907881
:1051E000309621F0208331834283538308959F3F7B
:1051F00031F0915020F4879577956795B795880F92
:10520000911D9695879597F90895DB018F939F934C
:105210000E949225BF91AF91A29F800D911DA39FE7
:10522000900DB29F900D11240895AA1BBB1B51E154
:1052300007C0AA1FBB1FA617B70710F0A61BB70B06
:10524000881F991F5A95A9F780959095BC01CD01AB
:10525000089597FB072E16F4009407D077FD09D028
:105260000E94152907FC05D03EF4909581959F4F2B
:105270000895709561957F4F0895DF93CF931F93A5
:105280000F939A9DF02D219FF00D8B9DF00D8A9D1F
:10529000E02DF10D039FF00D029FE00DF11D4E9DDD
:1052A000E00DF11D5E9DF00D4F9DF00D7F936F930E
:1052B000BF92AF925F934F93D5010E94FE258B0161
:1052C000AC01D7010E94FE25EB01E80FF91FD601C2
:1052D0000E948C292F913F91D6010E94FE25C60F76
:1052E000D71FE81FF91FAF91BF910E948C292F9102
:1052F0003F910E94FE25C60FD71FE81FF91FD60158
:105300000E94FE25E60FF71F9801BE01CF010F9105
:105310001F91CF91DF9108950E94FE25460F571FE0
:10532000C81FD91F08F431960895689401C0E89405
:10533000F92FF12B12F00C94C929A0E0B0E0E3EAB8
:10534000F9E20C94AB25092E059422F40E94252A3B
:10535000112392F4F0E80F26FFEFE094F09400950B
:105360001095B094C094D094A194BF0ACF0ADF0ADC
:10537000EF0AFF0A0F0B1F0B0E94D42907FC0E94A3
:10538000252ACDB7DEB7ECE00C94C725689401C0A0
:10539000E8948F929F92CF93DF930E94D429DF915C
:1053A000CF919F908F90089588249924F401E4016F
:1053B000B0E49F93AA279A158B049C04ED05FE0583
:1053C000CF05D007A10798F4AD2FDC2FCF2FFE2FEC
:1053D000E92D982C892E982F872F762F652F542F03
:1053E000432F322F2227B85031F7BF9127C01B2EF1
:1053F000BF91BB27220F331F441F551F661F771F06
:10540000881F991F881C991CEE1FFF1FCC1FDD1FD2
:10541000AA1FBB1F8A149B04EC05FD05CE05DF0502
:10542000A007B10748F08A189B08EC09FD09CE09CE
:10543000DF09A00BB10B21601A94E1F62EF4940160
:10544000AF01BE01CD01000C089560957095809567
:10545000909530954095509521953F4F4F4F5F4F18
:105460006F4F7F4F8F4F9F4F0895002E083090F061
:10547000982F872F762F652F542F432F322F2227D7
:105480000850F4CF220F331F441F551F661F771F8C
:10549000881F991F0A95B2F7002D089597FD109463
:1054A000002E083098F00850232F342F452F562F08
:1054B000672F782F892F912DF4CF15949795879585
:1054C0007795679557954795379527950A95AAF744
:1054D0001124002D08952A0D3B1D4C1D5D1D6E1DD0
:1054E0007F1D801F911F08952A193B094C095D09F2
:1054F0006E097F09800B910B08950024A7FD00948D
:105500002A17300540055005600570058005900597
:105510000895EE0FFF1F0590F491E02D09940F936D
:105520001F93CF93DF938230910510F482E090E0D7
:10553000E0917F04F091800430E020E0B0E0A0E052
:10554000309799F42115310509F44AC0281B390B0D
:1055500024303105D8F58A819B816115710589F167
:10556000FB0193838283FE0111C04081518102813E
:10557000138148175907E0F04817590799F4109715
:1055800061F012960C93129713961C933296CF01EA
:10559000DF91CF911F910F91089500937F04109395
:1055A0008004F4CF2115310551F04217530738F02C
:1055B000A901DB019A01BD01DF01F801C1CFEF01B3
:1055C000F9CF9093800480937F04CDCFFE01E20F4A
:1055D000F31F819391932250310939832883D7CFC8
:1055E00020917D0430917E04232B41F42091100101
:1055F0003091110130937E0420937D0420910E019F
:1056000030910F012115310541F42DB73EB740917E
:10561000120150911301241B350BE0917D04F09190
:105620007E04E217F307A0F42E1B3F0B281739075F
:1056300078F0AC014E5F5F4F2417350748F04E0FEE
:105640005F1F50937E0440937D04819391939FCF7D
:10565000F0E0E0E09CCFCF93DF930097E9F0FC010E
:10566000329713821282A0917F04B0918004ED01E1
:1056700030E020E01097A1F420813181820F931F48
:1056800020917D0430917E042817390709F061C00C
:10569000F0937E04E0937D04DF91CF910895EA01B9
:1056A000CE17DF07E8F54A815B819E014115510560
:1056B000B1F7E901FB83EA8349915991C40FD51FE2
:1056C000EC17FD0761F4808191810296840F951F8C
:1056D000E90199838883828193819B838A83F0E0A7
:1056E000E0E012968D919C9113970097B9F52D915A
:1056F0003C911197CD010296820F931F20917D045A
:1057000030917E042817390739F6309751F51092F9
:10571000800410927F04B0937E04A0937D04BCCFDC
:10572000D383C28340815181840F951FC817D90745
:1057300061F44E5F5F4F88819981480F591F5183F3
:1057400040838A819B81938382832115310509F0EF
:10575000B0CFF0938004E0937F049ECFFD01DC0185
:10576000C0CF13821282D7CFB0E0A0E0EAEBFBE219
:105770000C94A7258C01009751F4CB010E948F2A2D
:105780008C01C801CDB7DEB7E0E10C94C325FC0164
:10579000E60FF71F9C0122503109E217F30708F4C6
:1057A0009DC0D901CD91DC911197C617D70798F00C
:1057B000C530D10530F3CE0104978617970708F35B
:1057C000C61BD70B2297C193D1936D937C93CF01C6
:1057D0000E942B2BD6CF5B01AC1ABD0A4C018C0E5C
:1057E0009D1EA0917F04B0918004512C412CF12C7E
:1057F000E12C109731F580917D0490917E048815FD
:10580000990509F05CC04616570608F058C080910B
:105810000E0190910F01009741F48DB79EB7409112
:10582000120150911301841B950BE817F90708F03A
:1058300055C0F0937E04E0937D04F9017183608389
:10584000A0CF8D919C91119712966C901297139600
:105850007C901397A815B90559F56C0142E0C40E68
:10586000D11CCA14DB0420F1AC014A195B09DA012E
:105870001296159780F06282738251834083D9011A
:105880006D937C93E114F10471F0D7011396FC93AE
:10589000EE93129776CF22968C0F9D1FF90191837C
:1058A0008083F301EFCFF0938004E0937F0469CF0E
:1058B0004816590608F42C017D01D3019ACFCB017B
:1058C0000E948F2A7C01009749F0AE01B8010E9426
:1058D000792CC8010E942B2B870153CF10E000E0E8
:1058E00050CF9111089581568A5108F480528558FD
:1058F0000895FB01DC0102C001900D92415050401F
:10590000D8F70895FB01DC0101900D920020E1F72A
:105910000895FB01DC014150504030F08D91019021
:10592000801919F40020B9F7881B990B0895FB0121
:10593000DC014150504048F001900D920020C9F721
:1059400001C01D9241505040E0F7089511E0C0ECB5
:10595000D1E004C0FE010E94892A2196C13CD107F2
:10596000C9F7F894FFCF0101640016000000A040C1
:105970000000F04100008104800000000000A70248
:10598000EE013402F40265024302570200000000F7
:105990009A086D08C90833056608530844080000D2
:1059A00000003405EE01C90833059005A8051B0564
:1059B0000D0A00543D006F432000483D0025006F54
:1059C0004320413D006D0055563D003A00504D28A2
:1059D000312E302C322E352C3130293D00206E678F
:1059E0002F4C004C3D00206C782000424E4D4C3036
:1059F00033004E616E6F42326233504D00736572F8
:105A000069616C3A20002D35002D34002D33002DB6
:105A100032002D3100440056657273696F6E3A2072
:105A20000023007300534C20503D005061206973E7
:105A300020756E6C696B656C792100536561206C13
:105A40006576656C20503D00206850610055565ABF
:045A500000562000DC
:107E0000112484B714BE81FFF0D085E080938100F7
:107E100082E08093C00088E18093C10086E0809377
:107E2000C20080E18093C4008EE0C9D0259A86E02C
:107E300020E33CEF91E0309385002093840096BBD3
:107E4000B09BFECF1D9AA8958150A9F7CC24DD24C4
:107E500088248394B5E0AB2EA1E19A2EF3E0BF2EE7
:107E6000A2D0813461F49FD0082FAFD0023811F036
:107E7000013811F484E001C083E08DD089C08234E0
:107E800011F484E103C0853419F485E0A6D080C0E4
:107E9000853579F488D0E82EFF2485D0082F10E0AE
:107EA000102F00270E291F29000F111F8ED06801E7
:107EB0006FC0863521F484E090D080E0DECF843638
:107EC00009F040C070D06FD0082F6DD080E0C81688
:107ED00080E7D80618F4F601B7BEE895C0E0D1E017
:107EE00062D089930C17E1F7F0E0CF16F0E7DF06D8
:107EF00018F0F601B7BEE89568D007B600FCFDCFD4
:107F0000A601A0E0B1E02C9130E011968C91119780
:107F100090E0982F8827822B932B1296FA010C0160
:107F200087BEE89511244E5F5F4FF1E0A038BF0790
:107F300051F7F601A7BEE89507B600FCFDCF97BE46
:107F4000E89526C08437B1F42ED02DD0F82E2BD052
:107F50003CD0F601EF2C8F010F5F1F4F84911BD097
:107F6000EA94F801C1F70894C11CD11CFA94CF0C13
:107F7000D11C0EC0853739F428D08EE10CD085E9AC
:107F80000AD08FE07ACF813511F488E018D01DD067
:107F900080E101D065CF982F8091C00085FFFCCF94
:107FA0009093C60008958091C00087FFFCCF809118
:107FB000C00084FD01C0A8958091C6000895E0E648
:107FC000F0E098E1908380830895EDDF803219F02E
:107FD00088E0F5DFFFCF84E1DECF1F93182FE3DFCA
:107FE0001150E9F7F2DF1F91089580E0E8DFEE27F6
:047FF000FF270994CA
:027FFE00040479
:00000001FF
